:020000020000FC
:10000000FFC049C249C249C249C249C289C257C296
:1000100057C261C253C24FC24FC24FC241C241C256
:1000200049C27FC259C276C276C27CC278C276C249
:040030007AC27AC254
:10020000F89400E810E000936100109361000EE1A3
:1002100005B901E204B904E408B90FEB07B900E03D
:100220000BB90EEF0AB9B1E0A0E0D5E0C0E000E004
:100230000D93BD17E9F7AC17D9F714E00FEF1EBF08
:100240000DBF00E005BF03E00CBB07E005BB00E00D
:1002500004BD03E005BD00E006BD0AEF07BD0DEAE1
:1002600008BD00E003BD00E0009380000DE00093B6
:10027000810000E00093820010E000E01093850010
:10028000009384001CE10DE1109389000093880025
:1002900010E000E010938B0000938A0010E000E073
:1002A000109387000093860007E007BB00E00093EF
:1002B000B00000E00093B10000E00093B2000AEF4C
:1002C0000093B3000DEA0093B40000E00093B60081
:1002D00007E200937C0007EE00937A0000E00093B1
:1002E0007B0000E000937E0000E80093300000E017
:1002F00000937F0010E003E01093C5000093C4005A
:1003000000E20093C00008ED0093C10006E00093F6
:10031000C20000E000937B0000E000936900A89514
:1003200008E10093600009E20093600000E00093A0
:10033000640000E00DBB00E00093680000E0009363
:100340006B0000E000936C0000E000936D0004E09F
:1003500000936E0000E000936F0004E000937000D3
:1003600090E00DEA002EB1E0A0E20BE40093500112
:100370000CE40093510101E30093520107E3009361
:10038000530103E30093540102E50093550101E397
:100390000093560107E30093570103E300935801CC
:1003A00003E50093590100E300935A017894A8955E
:1003B00010E01C9B11601B9B1260103011F42EE4A6
:1003C0000CC0113011F422E608C0123011F429E7F4
:1003D00004C0133011F426EB00C0009178000091A6
:1003E0007900021718F002E3002E09C000E00016A1
:1003F000E9F30A9404C00DEA08BD0093B40020910B
:10040000520110915301009154018FD01A990AC0E2
:100410000D5A20F401951DEA010F04C01DEA101BBE
:10042000012F00C0009360010093B4002091560199
:10043000109157010091580178D019990AC00D5AAE
:1004400020F401951DEA010F04C01DEA101B012FC5
:1004500000C00093610108BD00915A010093620140
:10046000013311F4409A01C0409800E00093B200BB
:1004700004E005BB0091B10004600093B1005B98FB
:1004800000E006BD04E007BB05B5036005BD5D984F
:1004900004E1F7D08CCF18951895189518951895F4
:1004A0001895FFB60F935B9A05B5087F05BD0F91B0
:1004B000FFBE1895189518951895189518951895C4
:1004C000FFB60F935D9A0091B100087F0093B100D1
:1004D0000F91FFBE18951895FFB60F931F932F939A
:1004E0003F934F930091C6000B3411F4B1E0A0E2AA
:1004F000A03348F40D93AB3231F411E000E231E067
:1005000020E54BE094D04F913F912F911F910F9197
:10051000FFBE189518951895189518951895189563
:10052000189518951895189518953F93AF93BF9304
:10053000B0E0A0E02053203031F034E6A30F30E0EB
:10054000B31F2A95D1F71053103019F01A961A9547
:10055000E9F70053A00F00E0B01F1B2F0A2FBF9137
:10056000AF913F91089510E010937A0010917C00B4
:10057000107F102B10937C0000E000937B0005ECB3
:1005800000937A0000917A0006FDFCCF009178007C
:10059000109179000895011710F0201700F00895C8
:1005A0006F937F93712F602F621B730B28F0712F55
:1005B000602F461B570B00F07F916F9108954F936A
:1005C0005F936F934427552760E1000F111F441F6D
:1005D000551F4217530718F00395421B530B6A959A
:1005E000A1F75F934F932F913F916F915F914F913F
:1005F00008951F9317B5011708F0012F08BD1F912B
:1006000008951F931091B300011708F0012F009374
:10061000B4001F9108950F921F923F93019F112DD7
:10062000002D30E0CCDF3F911F900F900895AF93E5
:10063000BF93CF93DF93B12FA02FD32FC22F0D9154
:1006400009934A95E1F7DF91CF91BF91AF9108955A
:100650001F93F999FECF10E01FBB10E012BD81BDC2
:1006600000BD753A11F4FA9AF99A1F9108951F93F3
:10067000F999FECF10E012BD81BDF89A00B51F9127
:1006800008951F932F932BE11BE51A95F1F72A95F7
:0C069000D9F70A95C1F72F911F9108952A
:00000001FF
